:030000000211E406
:03000B000200C12F
:03002B000203CB02
:03005B0002051D7E
:0300730002051370
:1000800002030406080C10182030406080020304AC
:1000900006080C101820304080FF0406080C1018C9
:1000A0002030406080A0C000000001010003020277
:1000B000010D0D040506020D0505050D06030502DB
:1000C00002C2AFC0D0C0E0205A0D302F02E473301E
:1000D000600280F90203B7306306C286C291C295FE
:1000E00085258AC25AE525F4700221AA056130608F
:1000F00013206A19758B00D0E0D0D0C286C291C29D
:1001000095D2AF32C286C291C29502019AD26EC216
:100110006FE565601CC3E5611495654014C26ED23D
:100120006FC3E5619564500302019A756100020195
:100130009A206C14C286C291C295741AD5E0FDD281
:1001400090D292D29602019AC286C291C295E53DA2
:1001500020E22520E10D207502D290307502D29662
:1001600002019A20E005D29202019A207502D296ED
:10017000307502D29002019A20E11520E00D207521
:1001800002D290307502D29602019AD29202019A5E
:10019000207502D296307502D290758B00D0E0D0D7
:1001A000D0C286C291C295D2AF32D0E0D0D0D2AF09
:1001B0003261B7E525600A207502D286307502D219
:1001C00095C29161B7E5256002D291207502C29572
:1001D000307502C28661B7E525600A207502D295A6
:1001E000307502D286207502C286307502C29561D2
:1001F000B7207502C290307502C296E525600A20CC
:100200007502D286307502D295207502C29630757D
:1002100002C290C29161B7207502C290307502C2CD
:1002200096207502C296307502C290740ED5E0FD1C
:10023000E525600A207502D286307502D295C291FA
:1002400061B7207502C290307502C296E525600A3A
:10025000207502D286307502D295C292C29161B7E2
:10026000207502C290307502C296C292740ED5E01B
:10027000FDE525600A207502D286307502D295C24E
:100280009161B7C292E5256002D291207502C290B9
:10029000307502C296207502C295307502C2866121
:1002A000B7C292207502C290307502C296740ED504
:1002B000E0FDE5256002D291207502C295307502FD
:1002C000C28661B7C292E5256002D291207502C252
:1002D00096307502C290207502C295307502C286B2
:1002E00061B7C292207502C296307502C290740E38
:1002F000D5E0FDE5256002D291207502C2953075EA
:1003000002C28661B7207502C296307502C290E5BE
:1003100025600A207502D295307502D286C29220DD
:100320007502C286307502C29561B7207502C29609
:10033000307502C290C292740ED5E0FDE525600AC8
:10034000207502D295307502D286207502C28630A1
:100350007502C29561B7207502C296307502C290CF
:10036000E525600A207502D295307502D286207587
:1003700002C290307502C296207502C286307502A4
:10038000C29561B7207502C296307502C290207581
:1003900002C290307502C296740ED5E0FDE525606C
:1003A0000A207502D295307502D286207502C28667
:1003B000307502C29561B7E525F4F58A758B007535
:1003C0006000D25AD0E0D0D0D2AF32C2AFC0D0C0DD
:1003D000E0D2D3C2CEE528600A741F552E604915BD
:1003E00028812878007900E580307601F430E50234
:1003F00078FF53DACF20760343DA2030760343DAEE
:1004000010C2D8C269E580307601F430E50279FF88
:10041000C3E89970CE305903752818741F552E60A3
:10042000037528188858D268E52960041529813B8E
:10043000741F552E600543DA01C2D820680281CDB1
:10044000E558F8C268741F552E60367982B70431BA
:10045000C3E894F0400374F0F8E8C4540F28F87926
:1004600084B703028181C313C3138721200802C309
:0E04700013200A06C3C898F8818128F85003AB
:10047E0074FFF8C3E8955F5003E55FF8E52C54066A
:10048E00703D882230630AC3E522955C4003855C8B
:10049E00227882B60429C3E5229524401278A096CC
:1004AE00400DE52426F52450097524FF0204C0856D
:1004BE002224852425C3E524955C4003855C2520F4
:1004CE00CF09D0E0D0D0C2D3D2AF32C2CF7801E5BF
:1004DE00286008741F552E70021528C3E558940124
:1004EE004005755B0081FCE55B046002055BE55D24
:1004FE00C3240A5005755DFFA10AF55DD0E0D0D08A
:10050E00C2D3D2AF32C2AF53917FC258D2AF32C232
:10051E00AFC0D0C0E0C0F0D2D3A8FBA9FCC2D83087
:10052E006902A18053DACF20760343DA10307603C6
:10053E0043DA20D269E580307601F420E502A15439
:10054E0088268927E12053DACF20760343DA20303C
:10055E00760343DA10C2D8C269741F552E7002E1B9
:10056E00067800E580307601F430E502E106885821
:10057E00E10653DACF20760343DA2030760343DAEE
:10058E0010C269205902C13A53DACF20760343DAFA
:10059E001030760343DA20C2D8D26988538954C307
:1005AE00E89551F8E99552F9E4FB7AFAC3E894C854
:1005BE00E994005008E4D2E4FB7A0AC10DC3E89432
:1005CE0068E994015008E4D2E3FB7A0FC10DC3E849
:1005DE0094D0E994025008E4D2E2FB7A1EC10DC316
:1005EE00E894A0E994055008E4D2E1FB7A3CC10DF1
:1005FE00C3E89498E994085006E4D2E0FB7A78C3F5
:10060E00E89555FCE99556FD30E708ECF42401FC1D
:10061E00EDF4FD7557007008C3EC9A500375570141
:10062E0088558956A853A95488518952C3E89526EE
:10063E00F8E99527F9307402C1D9307302C1D93067
:10064E007202C1D2E9C313F9E813F8307102C1D2B4
:10065E00E9C313F9E813F8307002C1D2E9C313FDF0
:10066E00E813FC205918C3EC941CED9402400302CD
:10067E000706ED7009C3EC94C850030207207400FE
:10068E002077037896E624FAFEE43400FFC3EC9E4E
:10069E00FCED9FFD500678007900C1D9C3EC94FFA4
:1006AE00ED9400400678FF7900C1D9EC856CF0A47A
:1006BE00C5F0A2F733F8790040030206F578FF790A
:1006CE00000206F5E9C313F9E813F830740EE96079
:1006DE000278FFC3E81338F8E43400F9C3E894FF56
:1006EE00E99400400278FF8858D268205902E1064A
:1006FE00741FF4552E4BF52E752818741F552E7039
:10070E000375280A305902E120741F552E600353D9
:10071E00DAFE752906741F552E700375290AD0F05E
:10072E00D0E0D0D0C2D3D2AF327901E14F7903E11C
:10073E004F790AE14F791EE14F7964E14F79C8E1B3
:10074E004F7817E4D5E0FDD8FAD9F6227A147B78E3
:10075E000207767A107B8C0207767A0D7BB402073D
:10076E00767A0B7BC8020776AC257525017902B225
:10077E0075E4C292D5E0FDE5256002D291D5E0FD8B
:10078E00C291D5E0FDD292D5E0FDE525600A207537
:10079E0002D286307502D295E56DD5E0FD20750248
:1007AE00C286307502C2957496D5E0FDD9C1EAF8BD
:1007BE00D5E0FDD8FBDBB1C2928C2522C37C007D37
:1007CE000075F00005F0EA33FAEB33FB50F6EB134D
:1007DE00FBEA13FAC3E9FFE8FEE89AF8E99BF95041
:1007EE0004EFF9EEF8B3EC33FCED33FDD5F0DFEDAD
:1007FE00F9ECF822E889F08A20D2D4F8A9F07B002F
:10080E0030F70B7BFFF42401F8E9F43400F9E885A6
:10081E0020F0A4ADF0F8E98520F0A4AFF0FEED2EA7
:10082E00F974003FFA7C04C3EA13FAE913F9E813EA
:10083E00F8DCF48BF030F70AE8F42401F8E9F4342C
:10084E0000F9E889F0C2D4F8A9F0227882B6040340
:10085E000208B6C3E5589401400302087E8522249F
:0D086E00E4F53FF540F541F542F543F5484E
:10087B000208B67882E6FC754801E522F523783844
:10088B0079C7AA3BAB3CC3EB13FBEA13FAEC14603E
:10089B0013C3EB13FBEA13FAEC14146007C3EB134B
:1008AB00FBEA13FA1207CA883F894022E5486034F5
:1008BB00C3E53F9523F8E5409400F9500CC3E89449
:1008CB0080E994FF40160208EBC3E8947FE994009B
:1008DB0050030208EB787F79000208EB788079FFF0
:1008EB008844894522E5486058E5442541F8E545AB
:1008FB003542F9854520E4300701F43543FA30E7FA
:10090B0009C3EA94F0401502092DC3EA940F500372
:10091B0002092D78FF79FF7A0F02092D78007900F3
:10092B007AF0C3E524955C5006E52460092146E581
:10093B004520E70D2146E54530E706884189428A87
:10094B004322E54870030209B0789EE6FAC3E544FA
:10095B0033F8E54533F91102E930E70BC3E894802E
:10096B00E994FF40132187C3E8947FE99400500278
:10097B002187787F79002187788079FFE820E71538
:10098B00C3E52398F84009C3E8940140030209AE7C
:10099B0078010209AEE8F424012523F8400302098B
:1009AB00AE78FF884622E5487003020A12789FE66C
:1009BB00FAA842A9431102E930E70CC3E89401E914
:1009CB0094FF40160209E9C3E894FFE99400500331
:1009DB000209E978FF79000209E9780179FFE9203A
:1009EB00E715C3E54698F84009C3E89401400302B4
:1009FB000A107800020A10E8F424012546F8400397
:100A0B00020A1078FF8824227883E6F520120F5112
:100A1B0075E890E5E820ECF0A8BDA9BE120FE975CA
:100A2B006855756900C3740013FD745513FC745538
:100A3B002CFC74003DFDECFAEDFBC3E89AE99B40FE
:100A4B0014E5682455F568E5693400F569EA2CFA74
:100A5B00EB3DFB80E5AE68AF69C3E56913F9E5686B
:100A6B0013F8C3E913F9E813F8E56828F566E569A7
:100A7B0039F5677A03C3E913F9E813F8DAF7AA2013
:100A8B001A7009756800756900020AA71AEA6008EE
:100A9B00EE28FEEF39FFDAF88E688F692275E89041
:100AAB00227883E6FFE5E820ECF7A8BDA9BE056A2E
:100ABB00C3E56A94084052756A00E97007E56B60FC
:100ACB001B020ADBC3E8956B6010E56B5006600CEC
:100ADB0014020AE70460F9020AE7E56BF56BC394AD
:100AEB006DF84021755CC0C3E89404F84017755C41
:100AFB0080C3E89404F8400D755C40C3E89404F897
:100B0B004003755C0075BB0B22EFC39401601BC3E4
:100B1B00E894FFE994035012C3E89568E99569508E
:100B2B0009E55C600C155C020B3CE55CF4600205AE
:100B3B005CA85CC3E524985002A8248825C3E5254E
:100B4B00955D400B855D25E55DF46003855D5CC3BC
:100B5B00E56AB4070375BB1022306102783230624C
:100B6B00027878E52C5406601FE879A187F0A4C5BC
:100B7B00F0A2F733F8C3E8955C4002A85C882288A2
:100B8B00248825306102885E22788FE6FFC3EF94BC
:100B9B00055018C3EF94045020C3EF94035028C39F
:100BAB00EF94025030C3EF940150387533A0753475
:100BBB000F75353C75360561FC7533C07534127590
:100BCB00354075360661FC7533707534177535D045
:100BDB0075360761FC75334C75341D7535C4753628
:100BEB000961FC7533287534237535B875360B617F
:100BFB00FC85334F853450753B00753C0822A84F5C
:100C0B00A950020C14A849A94A759100C3E498F5A0
:100C1B0094E499F595759104D25875C820A8CCA980
:100C2B00CD75C824AA39AB3A8839893AC3E89AF802
:100C3B00E99BF9AA3BAB3CC3EB13FDEA13FCC3EDF9
:100C4B0013FDEC13FCC3EA9CFAEB9DFBEA28FAEBD1
:100C5B0039FB8A3B8B3C400122753BFF753CFF22E5
:0F0C6B00305802816B759100C3E4954BF594E40A
:100C7A00954CF595759104D258227892E6FF7E102C
:100C8A00305B027F053063047F037E00A93CA83BEA
:100C9A007A04C3E913F9E813F8DAF7C3E89EF8E926
:100CAA009400F94009C3E89402E9940050047802D8
:100CBA00E4F9E9FBE8FAC3E913FDE813FCC3EF948E
:100CCA0003602EEF20E00DE82CF8E93DF9ECFAED8F
:100CDA00FB020CE8E828F8E939F97A02E4FBC3EFE9
:100CEA009403400D8A4D8B4E8849894A8C4B8D4C12
:100CFA0022884D894E8A498B4A8C4B8D4C2230581A
:100D0A0002A108759100C3E4953BF594E4953CF57E
:100D1A0095759104D25822753E00752000020D3057
:100D2A00753E00752040D2AF053E20580122759DC0
:100D3A0000E53CC313C313F8086030306A06C313D6
:100D4A00C313F808C3E8940A4002780A306D08C34E
:100D5A00E8940440027804C3E53C9408400D759D6C
:100D6A0002C3E53C94104003759D03205803D2AF9B
:100D7A0022790F206D027905D2AF0000C2AF205A46
:100D8A000A7932206D027910306FE0306302797887
:100D9A00C3E58B9940D5E59BF4F45440B52002A1F4
:100DAA0030D8C8D2AF22C25B789CE6146007E53E11
:100DBA00147002D25B30630B053820581075380066
:100DCA00020DD72058071581158102173622759111
:100DDA0000C3E4954DF594E4954EF595759104D2CA
:100DEA005822AE25305B4F78A3E6FFBF010BD25CD9
:100DFA00752500C286C291C2959170305C03752533
:100E0A0000305802C105BF020BD25C752500C286AC
:100E1A00C291C29578A2B6010D9170305C03752516
:100E2A0000305802C125BF030BD25C752500C2866B
:100E3A00C291C295B1D8305C03752500305802C101
:100E4A0040305B04C25C8E2522C2AFC292206A0384
:100E5A00020E75900305206C12306E0F207502C2C7
:100E6A0096307502C290740ED5E0FD207502D290BC
:100E7A00307502D296759F56753D02D2AF22C2AF27
:100E8A00206A03020EAA9002C4306E17C29220751D
:100E9A0002C296307502C290740ED5E0FD020EAD04
:100EAA009001C5207502C295307502C286305A0675
:100EBA00E5256002D291207503759F76307503751A
:100ECA009F36753D03D2AF22C2AF207502C2903061
:100EDA007502C296206A03020EF4900283206C0AFD
:100EEA00306E07C292740ED5E0FD207502D296309C
:100EFA007502D290207503759F36307503759F76FB
:100F0A00753D04D2AF22C2AF206A03020F329002AB
:100F1A0042306E17207502C290307502C296C29294
:100F2A00740ED5E0FD020F359001B3C291305A0E0E
:100F3A00E525600A207502D286307502D295759F22
:100F4A0056753D05D2AF22C2AF207502C2963075E2
:100F5A0002C290206A03020F7B9001F1206C1230CA
:100F6A006E0F207502C290307502C296740ED5E0DB
:100F7A00FDD292207503759F76307503759F36757D
:100F8A003D06D2AF22C2AF206A03020FB9900356C0
:100F9A00306E1F207502C290307502C2962075020B
:100FAA00C296307502C290740ED5E0FD020FBC9055
:100FBA0001D7207502C286307502C295305A0EE5F5
:100FCA0025600A207502D295307502D286207503F3
:100FDA00759F36307503759F76753D01D2AF2290A5
:100FEA0001B1C286C291C295C290C292C29622C370
:100FFA00E54F9535E55095365001227890E6FFC3C6
:10100A00EF94055018C3EF9404501BC3EF94035098
:10101A001EC3EF94025021C3EF94015024C3E54F3D
:10102A00943CF8021054C3E54F9428F8021054C3B4
:10103A00E54F941AF8021054C3E54F9412F80210BF
:10104A0054C3E54F940AF8021054E5509400F98805
:10105A004F89502230580302105E22788076077832
:0F106A0081760778827601788476037883760121
:1010790078867609788F7601789076057895760264
:1010890078927603789B760D789376067887760141
:10109900789C760278887601788976017885760059
:1010A900788C7601788D7600788E76B47896762568
:1010B900789776D078987678789976C8789A7604F9
:1010C900789D7600227893E6FF756409756501C3FA
:1010D900BF0209756405756501021113C3BF0309D0
:1010E900756405756502021113C3BF0409756405AA
:1010F900756503021113C3BF050675640975650794
:10110900C3BF06067564007565007887E6FFC26C83
:10111900C3BF0302D26CC26BC3BF0402D26BC26AE3
:101129007418552D6002D26AC26E6002D26ED26FF7
:101139006002C26FC2757888E630E102D275C27664
:101149007889E630E102D276C3EF94026008758EA1
:1011590001D26D021164758E00C26D227880E61489
:1011690090008093789EF67881E6149000809378B9
:101179009FF6120FE922789BE61490008D9378A0D0
:10118900F6120FE9227886E61490009A9378A1F670
:10119900120FE922789CE6149000A79378A2F678BA
:1011A9009CE6149000AC9378A3F6120FE9222278FA
:1011B90096E6FA7897E6FB3077047A007BFFC3EB73
:1011C9009AFCC3948250027C82756C00056CEC8594
:1011D9006CF0A4C3E5F0948040F222C2D353D9BF86
:1011E9007581C043FF8012073775EF0243B203E5EB
:1011F900B324044002F5B37580BF75A44075F17C32
:1012090075D4DF75909875A56775F26775D5007502
:10121900A60175E241120FE9E4F8F6D8FD1165124D
:10122900176611CE3165317F318E319D31B731B8B5
:101239007898866D120FE975885075890275C824EA
:1012490075910475D84012074B12075A12074312B9
:101259000761120743120768120743121CE51207B8
:101269004B12074B12074775A82275B80275E6900D
:1012790075F610759B80759D0375D10E75BC5875F3
:10128900BB0B75BA1175E880120737D2AF120A1372
:1012990043DA01C2D8C26912074B753001D2597AB3
:1012A90005E55770027A0512073BE558C3940240D9
:1012B900EEE52E541F855A59F55AB559E2DAE2C2BC
:1012C9005953DACF20760343DA2030760343DA1014
:1012D900C2D8C26912074712073B7802741F552EFC
:1012E90070027800C3E5589840EDC2AF12075A1250
:1012F900075A12075AD2AF12074B75470012073B1C
:10130900788CE6C3940150030213CFE530C39401EE
:1013190050030213CF741F552E6035C3E55894FF4F
:1013290050030213CFC2AF12076FD2AF120747C3E0
:10133900E558940150EFC2AF12075A12073F12073E
:101349005AD2AF120747C3E55894FF40E9021D6A14
:101359007F05D27731B8120747C2AFC27731B8C318
:10136900E558947FD2AF4068C2AF12076FD2AFDFA2
:10137900E1C3E55894057897F612074B1218151230
:101389001CED7F0AD27731B8120747C2AFC2773155
:10139900B8C3E558947FD2AF50E8C2AF12075A12CA
:1013A900073F12075AD2AFDFDBE55824057896F6D6
:1013B90012074B121815121D1C120747C3E5589442
:1013C900FF40F6021D6AC3E5589547400385584713
:1013D900120747C3E558940140026106C2AF1207DC
:1013E9006F12076F12076FD2AF12074B753000E407
:1013F900F531F5320531E531F470360532789AE682
:101409007828146012785014600D78A01460087858
:10141900F0146003753200C3E53298401415327830
:1014290099866DC2AF12076FD2AF7898866D120791
:101439004712073BE5287008741F552E700241A614
:10144900C3E558940640AD120747E5287003021218
:10145900A6120FE9E4F522F523F524F525755CFFBD
:0E1469007885865FF53FF540F541F542F54385
:10147700F56AF548F52BF52CF55B120B94756A08A0
:1014870075BB10120737120AA8E5E820ECFBA8BDC8
:10149700A9BEE97001F8886B120AAC756A0875BBBA
:1014A700107895E630E0030214ED7887E6FE7602C1
:1014B70011CE7887EEF6D261C2AF120B6485225C3B
:1014C70085225DD2AFC26175250075620075630123
:1014D700D260D263753800120F51120F8F120C10A1
:1014E700120B9402161C7887E6FE76037893E6FDC6
:1014F700760511CE7887EEF67893EDF6D260D26155
:10150700D26E120F51120F8F120B64120737120E81
:1015170053120737120737120E8812073B120ED2E3
:1015270012073B12073B120F1012073F120F5112FF
:10153700073B120737C261D262120AA8120AAC121D
:101547000B64756A0875BB10120F8F120C09120C09
:1015570084120FF9115E120E53120C09120C841229
:101567000FF9115E120E88120C09120C84120FF972
:10157700115E120ED2120C09120C84120FF9115EB1
:10158700120F10120C09120C84120FF9115E120FB0
:1015970051120C09120C84120FF9C3E54F9535E56A
:1015A700509536400C115EC3E5589401508B0217D5
:1015B70036115EC2627887E6FE760211CE7887EE34
:1015C700F685225C855E5D855E2575620075630123
:1015D700D263753800C2AF207502C290307502C25F
:1015E70096207502C296307502C290742DD5E0FD23
:1015F700D2AF120F8F120C10120C6B120C84120D3B
:1016070008756A0075BB0B02161C11CE120F8F7579
:101617006A0075BB0B120D2A120DB0120DD81208F5
:1016270059120DEC120E53120C10120C6B120C8483
:10163700120D08120D21120DB0120DD81208B71293
:101647000DEC120E88120C10120C6B120C84120D7A
:1016570008120D2A120DB0120DD81208F0120DEC57
:10166700120ED2120C10120C6B120C84120D0812EF
:101677000D21120DB0120DD812094D120DEC120FDB
:1016870010120C10120C6B120C84120D08120D2A7A
:10169700120DB0120DD81209B1120DEC120F511222
:1016A7000C10120C6B120C84120D08120D21120A69
:1016B700A8120DB0120DD8120AAC120DEC120F8F32
:1016C700120C10120C6B120C84120D0830632A8551
:1016D7005E5C855E5D756200756301C3E538946481
:1016E700400AC263D264753714021700C3E55894E1
:1016F70001400302161C021736306419E5371470CF
:1017070005C264021611F537C3E558940140030278
:10171700161C021736C3E55B94FA5013741F552E37
:101727007004E5286009C3E53C94F05002C11C121F
:101737000FE97887E6FE760211CE7887EEF6E4F5B4
:1017470022F523F524F525F55FC260120737120F3E
:10175700E9741F552E7006E528700241A661F890BE
:101767001A0D7820121C00E520B4550CA3121C009A
:10177700E520B4AA03021787116512181502181479
:10178700901A037880121C00A308121C00A30812E9
:101797001C00901A067883121C00A308121C00A3D1
:1017A70008A308121C00A308121C00A308121C009F
:1017B700A308121C00A308A308A308121C00A3086F
:1017C700A308121C00A308121C00A308121C00A3E4
:1017D70008A308121C00A308121C00A308A30812E0
:1017E7001C00A308121C00A308121C00A308121C4B
:1017F70000A308121C00A308121C00A308121C0057
:10180700A308121C00A308121C00901A2122C2AFC1
:10181700121C3F121C19901A00740A121C05A3749B
:1018270004121C05A37410121C05901A0378801269
:101837001C04A308121C04A308121C04901A06789F
:1018470083121C04A308121C04A308A308121C0477
:10185700A308121C04A308121C04A308121C04A347
:0F18670008A308A308121C04A308A308121C045A
:10187600A308121C04A308121C04A308A308121C24
:1018860004A308121C04A308A308121C04A308122C
:101896001C04A308121C04A308121C04A308121C8F
:1018A60004A308121C04A308121C04A308121C0497
:0F18B600A308121C04121C52121C30901A21227B
:101A00000A04100909040103FF0901010155AA0193
:101A1000FFFF0105FF0306FF0225D02850040D0239
:021A200000FFC5
:101A4000235475726E6967794145333041232020F4
:101A500023424C48454C4923463333302320202031
:101A60002020202020202020202020202020202076
:101C0000E493F622E6438F01538FFD75EF0275B71B
:101C1000A575B7F1F0538FFE22438F02438F0175F4
:101C2000EF0275B7A575B7F1901A0DF0538FFC222E
:101C3000901A0D74559105901A0E74AA9105227A86
:101C40003079D07820901A409100E520F709A3DA86
:101C5000F7227A3079D0901A40E7910509A3DAF992
:101C600022AB6EA86FBB01057980021CE2BB0205A6
:101C70007981021CE2BB03057982021CE2BB0405E8
:101C80007984021CE2BB05057983021CE2BB0605D0
:101C90007995021CE2BB07057986021CE2BB0805A8
:101CA000798F021CE2BB09057990021CE2BB0A0590
:101CB0007992021CE2BB0B05799B021CE2BB0C056E
:101CC0007993021CE2BB0D057987021CE2BB0E056D
:101CD000799C021CE2BB0F057988021CE27989021B
:101CE0001CE2E8F7227C0512074BDCFB22C2AF1294
:101CF000075A12076112076812076F12073F12078F
:101D00005A12076112076812076F12073F12075A2B
:101D100012076112076812076FD2AF22C2AF120713
:101D20006F12076812076112075A12073F12076FF6
:101D300012076812076112075A12073F12076F1243
:101D4000076812076112075AD2AF22AE6EAF6FC298
:101D5000AF12075A12075A12075A12073FDEF21241
:101D6000076F12073FDFF8D2AF2291ED91E591E5C1
:101D7000756E01756F01757000B14B7C05AD581221
:101D8000074BC3ED955870F5C3E55894014009C35E
:101D9000E55894FF4032A1A6916112181591EDC249
:101DA000AF75EF1291E5DCD50570C3E57094035073
:101DB0000280C691E5056FE56E149000B193F808B6
:101DC000C3E56F98500280AE91E591E5056EC3E5DD
:101DD0006E94115002809C121065121815C2AF75D6
:041DE000EF1291E588
:00000001FF
